:020000040000FA
:020000000528D1
:08000800090083160313063002
:100010009F0083160313003085003F308600C030F8
:10002000870083120313FF308500FF308600FF3006
:100030008700831603138B018113011783120313A7
:1000400064002D28F8005539F9007808AA39F8001D
:100050000310F90D780C79040800FE30FD0005301E
:10006000FE007D0885000A30F500F50B35280608EE
:10007000222087000030F500F50B3C28FF30870078
:0A0080000314FD0DFE0B31282D289E
:02400E00723D01
:00000001FF
